:100000000C9434000C9451000C9451000C94510049
:100010000C9451000C9451000C9451000C942C0140
:100020000C9451000C9451000C9451000C94FB0062
:100030000C9451000C9451000C94CA000C94510083
:100040000C9451000C9451000C9451000C945100EC
:100050000C9451000C9451000C9451000C945100DC
:100060000C9451000C94510011241FBECFEFD8E026
:10007000DEBFCDBF11E0A0E0B1E0E8ECF7E002C0E8
:1000800005900D92A031B107D9F711E0A0E1B1E0E0
:1000900001C01D92A531B107E1F70E947A010C94CD
:1000A000E2030C940000CF92DF92EF92FF920F9345
:1000B0001F93CF93DF93EC01C880D980EA80FB8047
:1000C0002DEC3CEC4CEC5EE3C701B6010E940E0245
:1000D0000E94B3022DEC3CEC4CEC5EE30E945B030F
:1000E0009B01AC01C701B6010E94A90101E010E02B
:1000F0002DEC3CEC4CE45EE30E94570387FF02C00A
:1001000000E010E01D830C838E859F858230910571
:1001100061F08330910599F00197C9F416BC809184
:100120006E00826080936E0016C01092850010925F
:10013000840080916F00826080936F000CC01092E9
:10014000B2008091700082608093700004C081E0F2
:1001500090E00E94E20378949FB7F8948091120196
:100160009FBF8823C9F310921201EA85FB858C8119
:100170009D81892B19F08081846002C080818B7FF2
:100180008083DF91CF911F910F91FF90EF90DF90CF
:10019000CF9008951F920F920FB60F9211242F93B4
:1001A0003F938F939F93809110019091110101963D
:1001B000909311018093100180911201813091F090
:1001C000209110013091110180911301909114013F
:1001D0002817390738F081E080931201109211013D
:1001E000109210019F918F913F912F910F900FBE10
:1001F0000F901F9018951F920F920FB60F92112417
:100200002F933F938F939F938091100190911101B1
:100210000196909311018093100180911201813019
:1002200091F0209110013091110180911301909172
:1002300014012817390738F081E0809312011092D9
:100240001101109210019F918F913F912F910F906A
:100250000FBE0F901F9018951F920F920FB60F921E
:1002600011242F933F938F939F938091100190912E
:100270001101019690931101809310018091120158
:10028000813091F020911001309111018091130182
:10029000909114012817390738F081E080931201FA
:1002A00010921101109210019F918F913F912F9107
:1002B0000F900FBE0F901F901895FC0185B58360BD
:1002C00085BD21E030E0358724878AE090E0909377
:1002D00014018093130184B5826084BD89EF87BDCA
:1002E00037872687229A85E290E09387828780E08D
:1002F00090E00895CF92DF92EF92FF9280E091E03C
:100300000E945D01C12CD12C760160E070E0CB0130
:1003100060930001709301018093020190930301A7
:1003200080E091E00E9453008FEFC81AD80AE80AD3
:10033000F80AC701B6010E9476022FE632E143E0D7
:100340005BE30E945B0320E030E0A9010E94AA0168
:10035000DFCF5058BB27AA270ED058C149D130F063
:100360004ED120F031F49F3F11F41EF43EC10EF443
:10037000E095E7FB0BC1E92F5AD180F3BA1762076A
:1003800073078407950718F071F49EF589C10EF480
:10039000E0950B2EBA2FA02D0B01B90190010C0195
:1003A000CA01A0011124FF27591B99F0593F50F4AD
:1003B000503E68F11A16F040A22F232F342F442705
:1003C000585FF3CF469537952795A795F0405395FD
:1003D000C9F77EF41F16BA0B620B730B840BBAF0CD
:1003E0009150A1F0FF0FBB1F661F771F881FC2F738
:1003F0000EC0BA0F621F731F841F48F4879577954C
:100400006795B795F7959E3F08F0B3CF9395880F02
:1004100008F09927EE0F9795879508950CD0F6C0B0
:10042000EED040F0E5D030F021F45F3F19F0AEC0DF
:10043000511137C1DAC0FBD098F39923C9F3552382
:10044000B1F3951B550BBB27AA27621773078407C7
:1004500038F09F5F5F4F220F331F441FAA1FA9F37D
:1004600033D00E2E3AF0E0E830D091505040E6956F
:10047000001CCAF729D0FE2F27D0660F771F881FD0
:10048000BB1F261737074807AB07B0E809F0BB0BBF
:10049000802DBF01FF2793585F4F2AF09E3F5105E3
:1004A00068F074C0FEC05F3FECF3983EDCF38695C5
:1004B00077956795B795F7959F5FC9F7880F911D59
:1004C0009695879597F90895E1E0660F771F881F45
:1004D000BB1F621773078407BA0720F0621B730BF8
:1004E000840BBA0BEE1F88F7E0950895E89409C0D5
:1004F00097FB3EF490958095709561957F4F8F4F57
:100500009F4F9923A9F0F92F96E9BB279395F6956C
:10051000879577956795B795F111F8CFFAF4BB0FEA
:1005200011F460FF1BC06F5F7F4F8F4F9F4F16C04E
:10053000882311F096E911C0772321F09EE8872FD8
:10054000762F05C0662371F096E8862F70E060E094
:100550002AF09A95660F771F881FDAF7880F96950D
:10056000879597F9089585D080F09F3740F49111D1
:100570000EF097C060E070E080E89FEB089526F4ED
:100580001B16611D711D811D07C021C097F99F6752
:1005900080E870E060E00895882371F4772321F00B
:1005A0009850872B762F07C0662311F499270DC02A
:1005B0009051862B70E060E02AF09A95660F771FC5
:1005C000881FDAF7880F9695879597F908959F3FCA
:1005D00031F0915020F4879577956795B795880FFE
:1005E000911D9695879597F908959FEF80EC089552
:1005F00000240A9416161706180609060895002402
:100600000A9412161306140605060895092E03947B
:10061000000C11F4882352F0BB0F40F4BF2B11F4EF
:1006200060FF04C06F5F7F4F8F4F9F4F089557FD4E
:100630009058440F551F59F05F3F71F04795880F50
:1006400097FB991F61F09F3F79F0879508951216E7
:1006500013061406551FF2CF4695F1DF08C0161693
:1006600017061806991FF1CF869571056105089444
:100670000895E5DFA0F0BEE7B91788F4BB279F38DF
:1006800060F41616B11D672F782F8827985FF7CF73
:10069000869577956795B11D93959639C8F308951A
:1006A000E894BB2766277727CB0197F9089566D092
:1006B00008F48FEF08950BD0A9CF9ADF28F09FDFC1
:1006C00018F0952309F062CF90CF1124EACFAFDF65
:1006D000A0F3959FD1F3950F50E0551F629FF00155
:1006E000729FBB27F00DB11D639FAA27F00DB11DAE
:1006F000AA1F649F6627B00DA11D661F829F222737
:10070000B00DA11D621F739FB00DA11D621F839FBD
:10071000A00D611D221F749F3327A00D611D231F93
:10072000849F600D211D822F762F6A2F11249F57E1
:1007300050408AF0E1F088234AF0EE0FFF1FBB1F04
:10074000661F771F881F91505040A9F79E3F5105A3
:1007500070F01CCFA6CF5F3FECF3983EDCF386959C
:1007600077956795B795F795E7959F5FC1F7FE2B4E
:10077000880F911D9695879597F90895990F000810
:10078000550FAA0BE0E8FEEF16161706E807F90763
:10079000C0F012161306E407F50798F0621B730BFE
:1007A000840B950B39F40A2661F0232B242B252B7F
:1007B00021F408950A2609F4A140A6958FEF811D22
:0807C000811D0895F894FFCF9C
:1007C8000000000000000AD7233C000000000000E1
:00000001FF
